:020000040000FA
:06000000DBEF03F012002B
:0600080004EF04F01200F9
:060018000CEF04F01200E1
:02002A000000D4
:04002C000001776BED
:100030001E0E716E0401400E096F200E0A6F040E31
:100040000B6F880E086F0401200E0E6F040E0F6FE9
:10005000400E0C6F1200550EA76EAA0EA76EA68258
:1000600012000401226B010E236F12000001756B58
:10007000040121510001755D20E275C000F0016AA4
:10008000026A040122510024F36E23510120F46E10
:1000900024510220F86EF4CFF7FFF3CFF6FF0800EB
:1000A000F5CF76F000017551EA6A250FE96E040E6E
:1000B000EA2276C0EFFF752BDBD7F86A1200F00E4C
:1000C00004012217840EA66E0001756B04012151F4
:1000D0000001755D26E27551EA6A250FE96E040E8E
:1000E000EA22EFCF03F075C000F0016A026A040152
:1000F00022510024F36E23510120F46E245102207A
:10010000F86EF4CFF7FFF3CFF6FF03C0F5FF0C0056
:100110000F0E000175150F0801E19DDF0001752B21
:10012000D5D71200940EA66E0001756B0401215103
:100130000001755D1EE27551006E016A060ED890D1
:1001400000360136E804FBE1026A01BE02680401E0
:1001500022510024F36E23510120F46E2451022019
:10016000F86EF4CFF7FFF3CFF6FF75DF0001752BC4
:10017000DDD7F86A1200A66A0001756B04012151EF
:100180000001755D10E20401225100017525A96E80
:10019000A6807551EA6A250FE96E040EEA22A8CFFF
:1001A000EFFF752BEBD712000001756B0401215195
:1001B0000001755D15E20401225100017525A96E4B
:1001C0007551EA6A250FE96E040EEA22EF50A86E17
:1001D000040EA66E40DFA6B2FED70001752BE6D74F
:1001E0001200C40EA66E0001756B040121510001BE
:1001F000755D21E27551EA6A250FE96E040EEA2267
:10020000EFCF03F075C000F0016A026A04012251C9
:100210000024F36E23510120F46E24510220F86E65
:10022000F4CFF7FFF3CFF6FF03C0F5FF0C0013DFA9
:100230000001752BDAD7F86A1200060E00017A5D0C
:1002400003E36D50020B01E071D00001770511E16D
:1002500004010CBF0DD00401400E096F400E0401D3
:1002600008170401087D880E040108130001776B4C
:100270005DD0040108BF5AD00001756B0401205104
:10028000FF0A34E0F80A2DE0020A26E0010A1FE026
:10029000070A18E0010A11E0030A0AE0070A08E069
:1002A000060A01E032D0DDDE0001040E756F2ED0AB
:1002B000DDDE050E0001752729D001DF0001010EEA
:1002C000756F24D02FDF0001010E756F1FD053DF33
:1002D000050E000175271AD067DF0001010E756F4A
:1002E00015D07FDF0001010E756F10D06D960001F3
:1002F000786B796B00017807000E795B000178510B
:10030000791101E0F7D7FF0001D000D00001010E04
:10031000776F000175510AE075C00DF4400E0401BD
:0E0320000C1704010C7D880E04010C13120052
:02032E006C5011
:1003300002E0000E01D0010E00090BE004010051A3
:100340003C0BE842E8420D0802E1B2EF01F0BBEFDE
:1003500001F06C5002E0000E01D0010E040901E032
:1003600019D812000001606B616B666B676B90ECD3
:1003700002F03DEF02F0020E0001605D09E15CD881
:10038000040100BD02D0C80E01D0880E006F12001B
:1003900082EF02F0040E00017A5D09E112C46EFFE3
:1003A0006E50000802E2050E01D0030E7A6F0001C4
:1003B000600509E10AD8040104BD02D0C80E01D0CD
:1003C000880E046F120082EF02F00001080E665DD5
:1003D000000E675903E266C069F002D0080E696F2B
:1003E00069C005F46951006E016A0050665F0150F2
:1003F000675B180E646F040E656F69511CE00001A5
:100400007BA307D062C0F6FF63C0F7FF0800F5507A
:1004100005D062C0E9FF63C0EAFFEF5064C0E9FFA6
:1004200065C0EAFFEF6E0001622B000E6323642BB0
:1004300065236907E2D7120001C46AF000016A511E
:100440006625666F000E6721676F180E626F040ED7
:10045000636F6A5111E062C0E9FF63C0EAFFEF50C9
:1004600064C0E9FF65C0EAFFEF6E642B000E6523F0
:10047000622B63236A07EDD71200000161510BE183
:100480000401080E016F100E026F040E036F840E3C
:10049000006F040123D0040110AF22D00001665187
:1004A0000401165D000167510401175904E216C4E6
:1004B00066F017C467F089DF0001010E606F040168
:1004C000080E016F100E026F040E036F800E006F96
:1004D0000401180E066F040E076FC80E046F10D0CB
:1004E0000001020E606F0401056BC80E046F040169
:1004F000080E016F180E026F040E036FC80E006F16
:100500006D9812000001606B0401080E016F100E5F
:10051000026F040E036F880E006F0401046B12005B
:1005200004011051600BE842E842E842E842E84228
:10053000000901E012001151080A39E0010A35E012
:100540000F0A0AE0030A01E012000001010E616FC8
:100550000001040E7A6F12000001010E616F0401A8
:10056000130507E10001800E626F070E636F120E24
:1005700013D0020E135D07E10001920E626F070EA9
:10058000636F200E09D0030E135D0AE10001B20E65
:10059000626F070E636F040E0001666F676B02D017
:1005A0000001616B00017B831200E5EF02F00001A6
:1005B000010E616F00017C0E626F000E636F00011F
:1005C0007B930001010E666F12000001010E616F46
:1005D00012C47CF00401125104E10001050E7A6F8F
:0C05E00012000001060E7A6F16EF00F00A
:0405EC00080E6D6E1A
:1005F0006DBAFED7686A110E696E0001020E7A6F3D
:1006000012006850040B06E06950040B03E06D9281
:10061000699468946850010B04E06950010B01E093
:1006200027D86850100B09E06950100B06E0698468
:1006300068986D82A08A0300A19A6850200B09E097
:100640006950200B06E070A003D082EC02F070909D
:10065000689A030E00017A5D01E209D06850080B28
:1006600006E06950080B03E097EC01F06896120071
:10067000686A7B0E696E6E6A160E706E68A602D08E
:100680006896FCD76D9882EC02F000017C6B00014B
:06069000030E7A6F120058
:0A0696002A0EF66E000EF76E000E3D
:1006A000F86E00010900F550706F0900F550716F88
:1006B00003E1706701D03DD00900F5506B6F090070
:1006C000F5506C6F0900F5506D6F09000900F55089
:1006D000E96E0900F550EA6E090009000900F550BD
:1006E0006E6F0900F5506F6F09000900F6CF72F0C8
:1006F000F7CF73F0F8CF74F06BC0F6FF6CC0F7FF64
:100700006DC0F8FF00016E5302E16F5307E009006E
:10071000F550EE6E6E07F8E26F07F9D772C0F6FF7C
:1007200073C0F7FF74C0F8FF00017007000E715B23
:04073000BFD712001D
:0C073400A66AFE0EA96EA680A8CF7FF07A
:10074000FF0E00017F5D02E1000E01D0010E006E80
:100750008450080B01E0010E001402E000EF04F0E9
:100760008A9093908B9294928A808B82140E6F6EF3
:10077000F6EC02F001EC03F01DEC01F0FBD71200E7
:100780001201000200000008D8040BFF0000000066
:10079000000109022000010100803209040000026A
:1007A000000000000705010240000007058102402B
:0607B0000000040309042F
:0A07B60013EE00F023EE00F0F86AE5
:0E07C000059C4BEC03F09AEC03F0FDD7120001
:020000040030CA
:0100000024DB
:010001000EF0
:0100020028D5
:010003001EDE
:0100050000FA
:010006008178
:01000900C036
:01000B00A054
:00000001FF
